:100000000C942A001895000018950000189500001F
:10001000189500001895000018950000189500002C
:10002000189500000C94C40718950000189500005E
:10003000189500001895000018950000189500000C
:1000400018950000189500001895000018950000FC
:10005000189500008FE58DBFC4E0E0E84E2E88E0E3
:100060008EBFD8E0F7E05F2EEEEFF7E0A0E6B0E05D
:1000700088278D933197E9F7662481E48ABB81E371
:100080008BBB8FEB87BB8FEB88BB88E184BB83E0A6
:1000900085BB80E081BB8BE382BB80E08FBD81E0CC
:1000A0008EBD8FE181BD87E181BD86E086B980E4A8
:1000B00087B9C398C29AD89ADE9AC498C798C59847
:1000C000AC98F894A8950E94F3088091D3008062C0
:1000D0008093D300EFEFF1E0A4ECB0E091E00E9458
:1000E00031280091C400003081E009F080E08F9356
:1000F0000091C4000E3F80E010F009F081E09F9174
:10010000892B882311F40C9488008EEB8093C40013
:100110000091C4004AE0040F01BF89E190E00E9411
:10012000F426EAE0F0E0BB27A0E10E942E2801338C
:1001300011F40C94E300EAE0F0E0A0E1BB2781E3D6
:100140008C937BE70E941D28EBE0F0E0A0E1BB2749
:100150008FE08C937BE70E941D28ECE0F0E001E04B
:1001600010E0A0E1BB277BE70E941F28EEE0F0E053
:10017000A0E1BB2780E08C937BE70E941D28E2E191
:10018000F0E000E010E0A0E1BB277BE70E941F2821
:10019000EFE0F0E0A0E1BB2780E08C937BE70E94DA
:1001A0001D28E0E1F0E0A0E1BB2780E08C937BE735
:1001B0000E941D28E1E1F0E0A0E1BB2780E08C93E4
:1001C0007BE70E941D28EBE0F0E0AFEBB0E00E947F
:1001D0002E280091BF00043618F011F00C94F200A4
:1001E0000C94F50084E68093BF0080E797E9A0ECCB
:1001F000B0E08D939C93ECE0F0E0AAEBB0E00E94BD
:100200003028EEE0F0E0A5ECB0E00E942E28EFE010
:10021000F0E0A6ECB0E00E942E280E94F708E0E192
:10022000F0E0AFE6B0E00E942E28E1E1F0E0A0E7C8
:10023000B0E00E942E28E2E1F0E0A3E6B0E00E94E8
:100240003028A3E6B0E00E94F525E2E1F0E0A3E665
:10025000B0E07BE70E941F28AAEBB0E00D911C9153
:10026000003050E0150711F00C943C0181E090E063
:10027000AAEBB0E08D939C9380E08093D2008091B4
:100280006C00877F80936C0080E08093C80086E0DC
:100290008093C2008DE08093C300EBE6F0E0FA9318
:1002A000EA930E94D917229684E190E00E94F426F6
:1002B000DE980E94E026C49A88EC90E00E94F42622
:1002C000A89581B5886181BD877F81BDE0E6F0E0BA
:1002D000FA93EA930E94EF1B2296A8950091600082
:1002E000003011F40C947A010E94371B0E94BA0866
:1002F0000C947F018091D3008F7B8093D3000E9468
:10030000601B84E690E00E94F42600916B000030B0
:1003100018F011F00C948E010C949501EBE6F0E0CE
:10032000FA93EA930E94461922960027A3EDB0E0C3
:100330008C9186FB0EF401E040E0041711F00C9460
:10034000A3010E943C0F82E390E00E94F42678947F
:10035000A89581B5886081BD00916F00003011F0D3
:100360000C94B80181E090E0AAEBB0E08D939C93EF
:1003700000916F00013011F00C94CA01AAEBB0E0BB
:100380000D911C9141E050E0040F151FAAEBB0E065
:100390000D931C93A6EBB0E04D915C91AAEBB0E0FD
:1003A0000D911C910417150718F011F00C94DA0147
:1003B0000C94E00181E090E0AAEBB0E08D939C9377
:1003C0000027ACE6B0E08C9184FB0EF401E041E044
:1003D000041781E009F080E08F930027A3EDB0E0DF
:1003E0008C9186FB0EF401E040E0041781E009F0F7
:1003F00080E09F918923882311F40C941202EAEB88
:10040000F0E0FA93EA935A924A9280E0A42DB52D37
:100410008C9381E00E94E2250E94340D249681E0B5
:100420000E94DE2500917000023081E009F080E03A
:100430008F930027A3EDB0E08C9186FB0EF401E0D2
:1004400040E0041781E009F080E09F918923882330
:1004500011F40C944B0281B5886181BD877F81BD09
:10046000E3E0F0E00E946B26EAEBF0E0FA93EA9317
:100470005A924A9280E0A42DB52D8C9381E00E947F
:10048000E2250E94340D249681E00E94DE25A89585
:1004900081B5886081BD80E08093BC0080E080935E
:1004A0006B0080916C008F7780936C000027A3ED28
:1004B000B0E08C9186FB0EF401E041E0041711F0EE
:1004C0000C9464020E94F308A895ADE6B0E088277A
:1004D0008C930091D200003081E009F080E08F938E
:1004E0000027ACE6B0E08C9181FB0EF401E040E027
:1004F000041781E009F080E09F91892B882311F493
:100500000C94FE03E0E6F0E0FA93EA930E943118BF
:10051000229600916000003018F011F00C949202C5
:100520000C94FE0380916C00806880936C000091B5
:10053000D400003011F00C94EE024091C8000091FC
:100540006000041718F011F00C94A8020C94EE024D
:10055000809160008093C8000027ACE6B0E08C91E9
:1005600084FB0EF401E040E0041711F00C94C80283
:10057000A0E6B0E08C91AAEBB0E08D9388278C9335
:10058000ADE6B0E0E8EBF0E50E9436270C94EE0211
:100590000027A3EDB0E08C9187FB0EF401E041E071
:1005A000041711F00C94E802A0E6B0E00D911127B9
:1005B00041E050E0040F151FAAEBB0E00D931C932F
:1005C000ADE6B0E0E8EBF0E50E9436270C94EE02D1
:1005D000ADE6B0E0EAEBF0E50E9436270091D400EA
:1005E000013011F00C946E0300916000013011F0A5
:1005F0000C940003ADE6B0E0EAEBF0E50E9436278C
:1006000000916000023011F00C940C03ADE6B0E0F4
:10061000ECEBF0E50E94362780E0809362000091C9
:100620006000033081E009F080E08F930091BF000B
:10063000043681E008F080E09F918923882311F43B
:100640000C942A03AFEBB0E08C918E5F8C9381E029
:100650008093620000916000043081E009F080E046
:100660008F930091BF00023080E010F009F081E02C
:100670009F918923882311F40C944603AFEBB0E0DB
:100680008C9182508C9381E0809362000091620093
:10069000013011F00C946E038EB5887F8EBD5A9296
:1006A0004A928091BF00A42DB52D8C9381E00E94C9
:1006B000E2250E945122229681E00E94DE25EBE095
:1006C000F0E0AFEBB0E07BE70E941D280091D20084
:1006D000013011F00C946E0381E08EBD0091D400C6
:1006E000023011F00C94FE034091C80000916000AC
:1006F000041718F011F00C947F030C94FE03809102
:1007000060008093C80000916000013011F00C94EB
:10071000950381E090E0AAEBB0E08D939C93ADE669
:10072000B0E0E8EBF0E50E9436270091600002306F
:1007300011F00C94E603A6EBB0E00D911C91013092
:1007400050E0150718F011F00C94A8030C94E00386
:10075000A6EBB0E00D911C9141E050E0041B150B9D
:10076000A3E6B0E00D931C9301E010E00F931F93FC
:10077000A3E6B0E08D919C918A939A930E941026F3
:100780002296402F512F1F910F91040F151FA5E6A0
:10079000B0E00D931C93AAEBB0E04D915C91A5E6FF
:1007A000B0E00D911C910417150711F40C94B403DB
:1007B000A5E6B0E08D919C91AAEBB0E08D939C935F
:1007C000ADE6B0E0E8EBF0E50E943627009160006E
:1007D000033011F00C94F203ADE6B0E0EAEBF0E583
:1007E0000E94362700916000043011F00C94FE0343
:1007F000ADE6B0E0ECEBF0E50E9436270027ACE672
:10080000B0E08C9184FB0EF401E041E0041781E03C
:1008100009F080E08F930027A3EDB0E08C9187FB77
:100820000EF401E041E0041781E009F080E09F91BF
:1008300089238F930091D200013081E009F080E09C
:100840009F918923882311F40C946904AAEBB0E0EA
:100850000D911C91013050E0150711F00C946904C2
:10086000E0E6F0E0FA93EA930E94311822960091B4
:100870006000003080E010F009F081E08F93A6EB7B
:10088000B0E04D915C91A0E6B0E00D911127041706
:10089000150781E008F080E09F918923882311F4F7
:1008A0000C946904A0E6B0E00D91112741E050E0FE
:1008B000040F151FAAEBB0E00D931C93ADE6B0E05A
:1008C000E8EBF0E50E94362780916C008068809309
:1008D0006C000027ACE6B0E08C9180FB0EF401E0E8
:1008E00040E0041711F00C941A05EBE6F0E0FA93DF
:1008F000EA930E94D917229600916B00043011F000
:100900000C9489040E94AA0880916C0080688093EE
:100910006C0000916B00013011F00C949A04ADE66C
:10092000B0E0EAEBF0E50E94362780916C00806829
:1009300080936C0080E08093600000916B00023037
:1009400081E009F080E08F930091BF00043681E0E0
:1009500008F080E09F918923882311F40C94B80457
:10096000AFEBB0E08C918B5F8C9381E08093600063
:1009700000916B00033081E009F080E08F930091DB
:10098000BF00053081E009F080E09F918923882332
:1009900011F40C94D10481E08093BF0081E0809336
:1009A000600000916B00033081E009F080E08F93DC
:1009B0000091BF00053080E010F009F081E09F91C8
:1009C0008923882311F40C94ED04AFEBB0E08C91F3
:1009D00085508C9381E0809360000091600001302D
:1009E00011F00C941A058EB5887F8EBD5A924A92EA
:1009F0008091BF00A42DB52D8C9381E00E94E2254B
:100A00000E945122229681E00E94DE25EBE0F0E078
:100A1000AFEBB0E07BE70E941D280091D2000130CF
:100A200011F00C94150581E08EBD80916C008068FA
:100A300080936C00EDE6F0E0ADE6B0E00E94402768
:100A4000ADE6B0E08C91803081E009F480E08F93D6
:100A500000916B00003081E009F480E09F91892BC8
:100A60008F930091BC00013081E009F080E09F91FC
:100A7000892B882311F40C9456020091BC0001309C
:100A800011F00C94640580E08093BC00ADE6B0E00A
:100A9000EAEBF0E50E9436270027A3EDB0E08C9149
:100AA00087FB0EF401E041E0041711F00C9464059B
:100AB00081E090E0AAEBB0E08D939C93ADE6B0E0CE
:100AC000E8EBF0E50E943627ADE6B0E0E8EBF0E5B4
:100AD0000E94482811F00C94D6050091D2000130F4
:100AE00011F00C9475050E94AA08A6EBB0E04D9198
:100AF0005C91AAEBB0E00D911C910417150718F05A
:100B000011F00C94D1050027A3EDB0E08C9186FB89
:100B10000EF401E040E0041711F00C94A205EAEB9A
:100B2000F0E0FA93EA935A924A9280E0A42DB52D10
:100B30008C9381E00E94E2250E94340D249681E08E
:100B40000E94DE250027A3EDB0E08C9186FB0EF419
:100B500001E041E0041711F00C94CF050E94BA089F
:100B60000027A3EDB0E08C9186FB0EF401E040E09D
:100B7000041711F00C94CF05EAEBF0E0FA93EA9336
:100B80005A924A9280E0A42DB52D8C9381E00E9468
:100B9000E2250E94340D249681E00E94DE250C940B
:100BA000D40580E08093C8000C94F606EAEBF0E5EB
:100BB0000E94482811F00C946E060091D20001307A
:100BC00011F00C94E5050E94AA08AAEBB0E00E947F
:100BD000F5250027A3EDB0E08C9185FB0EF401E034
:100BE00041E0041711F00C940A060027ACE6B0E0CF
:100BF0008C9184FB0EF401E040E0041711F00C949A
:100C00000506AAEBB0E00E94FC258091D3008F7D01
:100C10008093D300A6EBB0E04D915C91AAEBB0E0DD
:100C20000D911C910417150718F011F00C941A0679
:100C30000C94200681E090E0AAEBB0E08D939C93A9
:100C40000027A3EDB0E08C9186FB0EF401E040E0BC
:100C5000041711F00C943F06EAEBF0E0FA93EA93E4
:100C60005A924A9280E0A42DB52D8C9381E00E9487
:100C7000E2250E94340D249681E00E94DE250027A3
:100C8000A3EDB0E08C9186FB0EF401E041E0041787
:100C900011F00C946C060E94BA080027A3EDB0E096
:100CA0008C9186FB0EF401E040E0041711F00C94E7
:100CB0006C06EAEBF0E0FA93EA935A924A9280E0EB
:100CC000A42DB52D8C9381E00E94E2250E94340D65
:100CD000249681E00E94DE250C94F606ECEBF0E50C
:100CE0000E94482811F00C94E6060091D2000130D1
:100CF00011F00C947D060E94AA08AAEBB0E00D91B9
:100D00001C91013050E0150718F011F00C948A0680
:100D10000C949006AAEBB0E00E94FC250C94980677
:100D2000A6EBB0E08D919C91AAEBB0E08D939C93E3
:100D30000027A3EDB0E08C9186FB0EF401E040E0CB
:100D4000041711F00C94B706EAEBF0E0FA93EA937B
:100D50005A924A9280E0A42DB52D8C9381E00E9496
:100D6000E2250E94340D249681E00E94DE250027B2
:100D7000A3EDB0E08C9186FB0EF401E041E0041796
:100D800011F00C94E4060E94BA080027A3EDB0E02D
:100D90008C9186FB0EF401E040E0041711F00C94F6
:100DA000E406EAEBF0E0FA93EA935A924A9280E082
:100DB000A42DB52D8C9381E00E94E2250E94340D74
:100DC000249681E00E94DE250C94F606EEEBF0E519
:100DD0000E94482811F00C94F606ECE0F0E0AAEB33
:100DE000B0E07BE70E941F280C94F60681E090E0BB
:100DF0000E94F4260027ACE6B0E08C9187FB0EF44D
:100E000001E040E0041718F011F00C9409070C946D
:100E1000C20700916B00003018F011F00C9412071B
:100E20000C947907A895E0E6F0E0FA93EA930E9423
:100E3000D917229600916000043011F00C946D07D0
:100E40000E94AA0880E08093C8000E94F50885E00F
:100E500090E00E94F42680E080936200E0E6F0E0FB
:100E6000FA93EA930E94D9172296A2E6B0E08C91F9
:100E70008F5F8C9388E090E00E94F42600916000E0
:100E8000003081E009F080E08F9300916200043629
:100E900080E010F009F081E09F91892B882311F404
:100EA0000C942E0700916200043618F011F00C9497
:100EB0005B070C946A0781B5886181BD877F81BD1E
:100EC000E3E6F0E0FA93EA930E94AC09229681B53A
:100ED000886081BD80E08093600081E090E00E94A6
:100EE000F42600916000003011F00C9412070C946D
:100EF000B8070091D400013011F00C94B40780E0E1
:100F000090E0A3E6B0E08D939C93E0E6F0E0FA93E6
:100F1000EA930E9431182296A3E6B0E00E94F525DC
:100F2000EF93FF93ECE8F1E00E94C826FF91EF9168
:100F300000916000003081E009F080E08F93A3E62B
:100F4000B0E00D911C91083250E0150780E010F0E0
:100F500009F081E09F91892B882311F40C94850777
:100F600081E090E00E94F42681E090E00E94F42667
:100F70000091D200003011F00C94C20785E090E09F
:100F80000E94F4260C9451020F921F922F923F92CE
:100F90004F925F927F92AF92BF920F931F932F93C6
:100FA0003F934F935F936F937F938F939F93AF93F1
:100FB000BF93CF93DF93EF93FF938FB78F93F89403
:100FC00089B78B7F89BF8EB5887F8EBD5A924A9232
:100FD00080E092E0A42DB52D8D939C9382E00E9439
:100FE000E2250E945C25229682E00E94DE25009187
:100FF000DD000A3011F00C94FF070E94F3080E94F4
:10100000CD1E0091DD000A3011F00C940C080E94F6
:10101000F50880E08093DD00ADEDB0E08C918F5F4E
:101020008C93A8950027A3EDB0E08C9186FB0EF47D
:1010300001E040E0041711F00C9431085A924A92F2
:1010400080E092E0A42DB52D8D939C9382E00E94C8
:10105000E2250E945C25229682E00E94DE250E9405
:10106000CD1EA9EDB0E04D915D916D917C91A5ED06
:10107000B0E00D911D912D913C910E94942780E04C
:101080000CF481E08F930027A3EDB0E08C9186FBF8
:101090000EF401E040E0041781E009F080E09F9148
:1010A0008923882311F40C94620880E49CE99093CE
:1010B0004D0080934C0081E08EBD89B7846089BF6C
:1010C0000C948C0880E08093D20080916C00877F24
:1010D00080936C000027A3EDB0E08C9186FB0EF4AA
:1010E00001E040E0041711F00C947F08ACE6B0E09A
:1010F0008C9184FBACEBB0E0882780F98C93009155
:10110000C5004FE70423A1E6B0E00C930E94F50868
:1011100080E08093C800AC988F918FBFFF91EF91D2
:10112000DF91CF91BF91AF919F918F917F916F91FF
:101130005F914F913F912F911F910F91BF90AF9071
:101140007F905F904F903F902F901F900F90189539
:10115000F894FFCF89B78B7F89BF8EB5887F8EBD0E
:1011600080E08093D20080916C00877F80936C0038
:10117000AC980895DE9A6E98C498C598C7980E9456
:10118000F508E2E0F0E00E946B26DE98C49A0E9427
:10119000E02684E690E00E94F426A8958091D30092
:1011A0008F7B8093D300E0E6F0E0FA93EA930E940D
:1011B000EF1B229600916000003011F40C94F008AF
:1011C0008091D30080648093D30084E690E00E94F5
:1011D000F426DE9A6E98C498C598C7980C94F208C5
:1011E0000E943C0F0895AB980895AB9A089581E052
:1011F0000E94032780916C008F7E80936C00009189
:10120000C50041E00423A881B9810C93A881B9816C
:101210000C91003011F40C94120980916C008061E3
:1012200080936C008091D3008F778093D3000091DE
:10123000C50042E00423A881B9810C93A881B9813B
:101240000C91003011F40C942A098091D30080682D
:101250008093D30080916C008E7F80936C0000910E
:10126000C50044E00423A881B9810C93A881B98109
:101270000C91003011F40C94420980916C00816053
:1012800080936C0080916C008D7F80936C00009146
:10129000C50048E00423A881B9810C93A881B981D5
:1012A0000C91003011F40C945A0980916C0082600A
:1012B00080936C0080916C008F7D80936C00009116
:1012C000C50040E20423A881B9810C93A881B981AB
:1012D0000C91003011F40C94720980916C008062C2
:1012E00080936C008091D3008F7E8093D300009117
:1012F000C60041E00423A881B9810C93A881B9817B
:101300000C91003011F40C948A098091D300806113
:101310008093D3000091C60046E00423A881B981E0
:101320000C93A881B9810C9142E00E9438280C935B
:10133000A881B9818C918093D4000091D4000330AE
:1013400011F00C94A60982E08093D40081E0481A41
:101350008827580A2296089582E00E94032781E098
:101360000E94032781E00E94032780E0AA81BB81BD
:101370008C9383E4A0EAB0E08C938FE4A1EAB0E020
:101380008C938EE4A2EAB0E08C9386E4A3EAB0E00A
:101390008C9389E4A4EAB0E08C93ACE6B0E08C9145
:1013A00085FBA881B981882780F98C9380916C0096
:1013B000806280936C00A6E7B0E00D911D912D91A5
:1013C0003C91A6E9B0E00D931D932D933C935A9266
:1013D0004A92A6E9B0E00D911D912D913C91A42D6A
:1013E000B52D0D931D932D933C9384E00E94E2252F
:1013F0005A924A9280E090E0A42DB52D8D939C9353
:1014000082E00E94E2255A924A9281E0A42DB52DF5
:101410008C9381E00E94E2250E944B10269687E083
:101420000E94DE258FE00E940327E8EAF0E006E054
:10143000A881B9810E940F28A881B981E0ECF0E56C
:101440000E9448280FB68FE0481A8827580A22962B
:101450000FBE81E009F080E08F9300919100003190
:1014600081E009F080E09F918923882311F40C9496
:10147000870A81E0AA81BB818C93A6E9B0E00D9137
:101480001D912D913C91A6E7B0E00D931D932D93F6
:101490003C9380916C008F7D80936C005A924A92AD
:1014A000A6E9B0E00D911D912D913C91A42DB52D93
:1014B0000D931D932D933C9384E00E94E2255A9254
:1014C0004A9280E090E0A42DB52D8D939C9382E00C
:1014D0000E94E2255A924A9280E0A42DB52D8C9369
:1014E00081E00E94E2250E944B10269687E00E9430
:1014F000DE25A6E9B0E00D911D912D913C91A6E766
:10150000B0E00D931D932D933C930E94E10AA881B6
:10151000B9818C9180FBACE6B0E08C9185F98C931D
:10152000AAE7B0E00D911D912D913C91A6E7B0E0A6
:101530000D931D932D933C93A6E7B0E00D911D9163
:101540002D913C91A6E9B0E00D931D932D933C9312
:101550005A924A92A6E9B0E00D911D912D913C91CD
:10156000A42DB52D0D931D932D933C9384E00E94E3
:10157000E2255A924A9280E090E0A42DB52D8D93F9
:101580009C9382E00E94E2255A924A9280E0A42D28
:10159000B52D8C9381E00E94E2250E944B10269687
:1015A00087E00E94DE25AA81BB818C91AE81BF813C
:1015B0008D9388278C9384E0481A8827580A2696AA
:1015C000089582E00E94032781E00E94032781E0C2
:1015D0000E940327789481E090E0AC81BD818D93D7
:1015E0009C93EA81FB81FA93EA93EE81FF81FA935F
:1015F000EA930E94F70C2496AA81BB810C910130DA
:1016000011F00C940E0B82E090E0AC81BD818D93C3
:101610009C9381E08093C5000C942A0B023011F05A
:101620000C941D0B83E090E0AC81BD818D939C9365
:1016300080E08093C5000C942A0B033011F00C94C9
:101640002A0B84E090E0AC81BD818D939C9383E074
:101650008093C500EEE0F0E0A5ECB0E07BE70E94EF
:101660001D28EC81FD81FA93EA935A924A9280E018
:10167000A42DB52D8C9381E00E94E2250E94340DAB
:10168000249681E00E94DE250091D200003011F006
:101690000C94440B88EC90E00E94F42685E090E0E6
:1016A000AC81BD818D939C93EA81FB81FA93EA938F
:1016B000EE81FF81FA93EA930E94F70C2496EEE004
:1016C000F0E0A5ECB0E00E942E28AA81BB810C912D
:1016D000033011F00C946E0B0C940B0CAA81BB819F
:1016E0000C91013011F00C947C0BA5ECB0E08C91C6
:1016F00088608C930C94850B023011F00C94850B50
:10170000A5ECB0E08C91877F8C93EEE0F0E0A5EC47
:10171000B0E07BE70E941D2888EC90E00E94F42650
:1017200086E090E0AC81BD818D939C93EA81FB8142
:10173000FA93EA93EE81FF81FA93EA930E94F70C01
:101740002496AA81BB810C91033011F00C94AA0B52
:101750000C940B0CEEE0F0E0A5ECB0E00E942E281B
:10176000AA81BB810C91013011F00C94BE0BA5EC49
:10177000B0E08C9184608C930C94C70B023011F014
:101780000C94C70BA5ECB0E08C918B7F8C93EEE0B2
:10179000F0E0A5ECB0E07BE70E941D2888EC90E02B
:1017A0000E94F42687E090E0AC81BD818D939C93EC
:1017B000EA81FB81FA93EA93EE81FF81FA93EA933F
:1017C0000E94F70C2496EEE0F0E0A5ECB0E00E9459
:1017D0002E28AA81BB810C91013011F00C94F70BDB
:1017E000A5ECB0E08C9180628C930C94000C0230DC
:1017F00011F00C94000CA5ECB0E08C918F7D8C93D3
:10180000EEE0F0E0A5ECB0E07BE70E941D2888EC5C
:1018100090E00E94F42688E090E0AC81BD818D9339
:101820009C93EC81FD81FA93EA930E94D50C229659
:101830000091C50043E00423A881B9810C93A881DD
:10184000B9810C91003011F00C942E0C83E090E0E3
:10185000AC81BD818D939C930C94440C013011F0AC
:101860000C943A0C82E090E0AC81BD818D939C9306
:101870000C94440C033011F00C94440C84E090E080
:10188000AC81BD818D939C93EC81FD81FA93EA93A9
:101890000E94D50C22960091C50048E00423A8813F
:1018A000B9810C93A881B9810C91003011F00C948E
:1018B000610C8AE090E0AC81BD818D939C930C9487
:1018C0006B0C083011F00C946B0C89E090E0AC814B
:1018D000BD818D939C93EC81FD81FA93EA930E94E4
:1018E000D50C22960091C50044E00423A881B9815B
:1018F0000C93A881B9810C91003011F00C94880CE4
:101900008BE090E0AC81BD818D939C930C94920C04
:10191000043011F00C94920C8CE090E0AC81BD810D
:101920008D939C93EC81FD81FA93EA930E94D50CF0
:1019300022960091C50040E20423A881B9810C934E
:10194000A881B9810C91003011F00C94AF0C8DE09E
:1019500090E0AC81BD818D939C930C94B90C0032C6
:1019600011F00C94B90C8EE090E0AC81BD818D93A8
:101970009C93EC81FD81FA93EA930E94D50C229608
:101980008FE090E0AC81BD818D939C93EC81FD81D3
:10199000FA93EA930E94D50C22960E94F70884E0FD
:1019A000481A8827580A26960895E881F981FA93FB
:1019B000EA935A924A9280E0A42DB52D8C9381E04F
:1019C0000E94E2250E94340D249681E00E94DE25CB
:1019D00082E390E00E94F4260091D200003011F0E2
:1019E0000C94EC0C82E390E00E94F426089581E0D0
:1019F0000E940327EA81FB81FA93EA935A924A9262
:101A000080E0A42DB52D8C9381E00E94E2250E94F8
:101A1000340D249681E00E94DE2584E690E00E9449
:101A2000F426E881F981FA93EA930E94D917229665
:101A3000A881B9810C91003018F011F00C94220D9E
:101A40000C94110D0E94AA0884E190E00E94F426F3
:101A5000A881B9818C91AC81BD818C9381E0481AB9
:101A60008827580A2296089582E00E94032781E081
:101A70000E9403278EB5887F8EBD80916C00877F82
:101A800080936C00A6E7B0E00D911D912D913C91E3
:101A9000A6E9B0E00D931D932D933C935A924A9280
:101AA000A6E9B0E00D911D912D913C91A42DB52D8D
:101AB0000D931D932D933C9384E00E94E2255A924E
:101AC0004A92AA85BB858D919C91A42DB52D8D93AD
:101AD0009C9382E00E94E2255A924A9280E0A42DD3
:101AE000B52D8C9381E00E94E2250E944B10269632
:101AF00087E00E94DE2540E050E060E070E0A2E96F
:101B0000B0E00D911D912D913C910E94942711F010
:101B10000C948C0D0C94360FAC9A0E9405225A92AC
:101B20004A928091BF00A42DB52D8C9381E00E9434
:101B3000E2250E945122229681E00E94DE255A92DF
:101B40004A92A0ECB0E08D919C91A42DB52D8D937F
:101B50009C9382E00E94E2250E94E922229682E084
:101B60000E94DE25A6E9B0E00D911D912D913C91DA
:101B7000A5EDB0E00D931D932D933C93A6E9B0E045
:101B80000D911D912D913C91A2E9B0E04D915D9197
:101B90006D917C910E948A27A9EDB0E00D931D9371
:101BA0002D933D9380E0A881B9818C930E94CD1E36
:101BB00081E090E0AA81BB818D939C93AA81BB8137
:101BC0000D911C910F3F51E0150718F011F00C9486
:101BD000180EAA81BB81AD90BC90ADEDB0E0AA0D0E
:101BE000BB1D0C910F3F81E009F080E08F93AA812B
:101BF000BB81AD90BC90AEEDB0E0AA0DBB1D0C91C9
:101C00000F3E80E010F009F081E09F918923882346
:101C100011F40C94110E81E0A881B9818C930C947D
:101C2000180EAA81BB810E94F52510F40C94DE0DDC
:101C3000A881B9810C91013011F00C94D60DAA81C4
:101C4000BB81AD90BC90AFEDB0E0AA0DBB1D8C91F7
:101C5000AA81BB818D9388278C93AA81BB810D912A
:101C60001C9140E150E00E944A26AA81BB814D931D
:101C70005C9380E18093C700AA81BB810D911C9188
:101C8000013050E0150711F00C944B0E84E0809366
:101C9000C7000C94D80E023050E0150711F00C94D8
:101CA000560E85E08093C7000C94D80E033050E0A8
:101CB000150711F00C94610E86E08093C7000C9418
:101CC000D80E043050E0150711F00C946C0E87E02C
:101CD0008093C7000C94D80E053050E0150711F022
:101CE0000C94770E88E08093C7000C94D80E0630D1
:101CF00050E0150711F00C94820E8AE08093C70023
:101D00000C94D80E073050E0150711F00C948D0E8E
:101D10008CE08093C7000C94D80E083050E0150773
:101D200011F00C94980E8EE08093C7000C94D80E9E
:101D3000093050E0150711F00C94A30E80E1809358
:101D4000C7000C94D80E0A3050E0150711F00C941F
:101D5000AE0E84E18093C7000C94D80E0B3050E097
:101D6000150711F00C94B90E88E18093C7000C940C
:101D7000D80E0C3050E0150711F00C94C40E8CE115
:101D80008093C7000C94D80E0D3050E0150711F069
:101D90000C94CF0E80E28093C7000C94D80E0E30C6
:101DA00050E0150711F00C94D80E88E28093C7001C
:101DB000A2E9B0E00D911D912D913C9140E052E0DF
:101DC00060E070E00E941327A7E6B0E00D931D933A
:101DD0002D933D93A7E6B0E00D911D912D913C917F
:101DE000A7ECB0E04C915527662777270E94742610
:101DF000A7E6B0E04D935D936D937D93A7E6B0E0C9
:101E00000D911D912D913C9148EE53E060E070E002
:101E10000E947426A7E6B0E04D935D936D937D9389
:101E2000AC81BD810C91003011F00C94360F009103
:101E30006F00013011F00C94240FECE0F0E0AAEBFD
:101E4000B0E07BE70E941F2881E08093D20088ECFD
:101E50009FEA90934D0080934C0089B7846089BFBE
:101E600081E08EBD85E090E00E94F42683E0481A70
:101E70008827580A24960895A895A6E7B0E00D9102
:101E80001D912D913C91AAE7B0E00D931D932D93E8
:101E90003C93A6E7B0E00D911D912D913C91A6E9F0
:101EA000B0E00D931D932D933C935A924A92A6E96C
:101EB000B0E00D911D912D913C91A42DB52D0D9368
:101EC0001D932D933C9384E00E94E2255A924A92FE
:101ED00080E090E0A42DB52D8D939C9382E00E942C
:101EE000E2255A924A9280E0A42DB52D8C9381E090
:101EF0000E94E2250E944B10269687E00E94DE2574
:101F0000A895A6EBB0E00D911C91013050E01507AB
:101F100010F00C94B20F5A924A9281E0A42DB52D84
:101F20008C9381E00E94E2250E944323229681E067
:101F30000E94DE258CE291E00E94F4265A924A9299
:101F400080E0A42DB52D8C9381E00E94E2250E94B3
:101F50004323229681E00E94DE258091D300806495
:101F60008093D300A895A6E7B0E00D911D912D9127
:101F70003C91A6E9B0E00D931D932D933C93AAEB01
:101F8000B0E00D911C91003050E0150781E009F0A0
:101F900080E08F93A6EBB0E04D915C91AAEBB0E0AE
:101FA0000D911C910417150780E010F009F081E0F5
:101FB0009F91892B882311F40C94E40F81E090E029
:101FC000AAEBB0E08D939C930E94F508089584E0FD
:101FD0000E940327A5EDB0E00D911D912D913C913C
:101FE000A881B9810D931D932D933C93A6E7B0E092
:101FF0000D911D912D913C91A6E9B0E00D931D939B
:102000002D933C935A924A92A6E9B0E00D911D910E
:102010002D913C91A42DB52D0D931D932D933C93A3
:1020200084E00E94E2255A924A928FE19EE4A42D18
:10203000B52D8D939C9382E00E94E2255A924A929C
:1020400080E0A42DB52D8C9381E00E94E2250E94B2
:102050004B10269687E00E94DE25A6E7B0E00D91A2
:102060001D912D913C91A6E9B0E00D931D932D9308
:102070003C93A881B9810D911D912D913C91A5EDC5
:10208000B0E00D931D932D933C9384E0481A88276C
:10209000580A2296089581E00E94032781E00E9459
:1020A000032781E00E94032780E090E0A8EBB0E0E6
:1020B0008D939C9380916C008F7B80936C0000E0EB
:1020C00010E020E030E0A2E9B0E00D931D932D93E5
:1020D0003C930027ACE6B0E08C9185FB0EF401E068
:1020E00041E0041781E009F080E08F93A885B9856D
:1020F0000D911C91003050E0150781E009F480E05B
:102100009F9189238F93AE81BF810C91003081E034
:1021100009F080E09F918923882311F40C94EB103F
:10212000AAE9B0E0E885F9850E94A727EAE9F0E08E
:10213000A8E6B7E00E940328E8E6F7E0AAE9B0E0E5
:102140001127222704E033270E944C2781E4AC8129
:10215000BD818C93AC81BD818C918093A00081E086
:10216000EAE9F0E001E00A93ADE6B0E00E94082859
:10217000ADE6B0E08C91A1EAB0E08C9382E0EAE9B0
:10218000F0E001E00A93ADE6B0E00E940828ADE679
:10219000B0E08C91A2EAB0E08C9383E0EAE9F0E051
:1021A00001E00A93ADE6B0E00E940828ADE6B0E099
:1021B0008C91A3EAB0E08C9384E0EAE9F0E001E0DE
:1021C0000A93ADE6B0E00E940828ADE6B0E08C913D
:1021D000A4EAB0E08C9389B78B7F89BF8EB5887FE6
:1021E0008EBD81B5886181BD877F81BDAEECB0E0D9
:1021F0000D911D912D913C91AAECB0E00D931D9392
:102200002D933C93AAE7B0E04D915D916D917C9147
:10221000A6E7B0E00D911D912D913C910E9494276D
:1022200011F00C941D1102E010E020E030E0AAEC67
:10223000B0E00D931D932D933C9380E0A881B9816C
:102240008C93EA81FB81FA93EA935A924A92AE8583
:10225000BF850D911D912D913C91A42DB52D0D9310
:102260001D932D933C9384E00E94E2250E949620CA
:10227000249684E00E94DE25AA81BB810C910E3F4A
:1022800011F40C944F118091D30080648093D3009B
:1022900080916C00806480936C000C9462115A925F
:1022A0004A92AA85BB858D919C91A42DB52D8D93C5
:1022B0009C9382E00E94E2250E946512229682E0B1
:1022C0000E94DE25A881B9818C918F5F8C9340910B
:1022D0007300A881B9810C91041781E009F080E0B6
:1022E0008F930027ACE6B0E08C9186FB0EF401E002
:1022F00041E0041781E009F480E09F91892388235D
:1023000011F40C941812009182000B3011F00C940F
:10231000C511EAECF0E0FA93EA935A924A92AAECD9
:10232000B0E00D911D912D913C91A42DB52D0D93F3
:102330001D932D933C9384E00E94E2250E947D161C
:10234000249684E00E94DE25EA85FB85FA93EA93D1
:102350005A924A92AAECB0E00D911D912D913C91B8
:10236000A42DB52D0D931D932D933C9384E00E94D5
:10237000E2250E941316249684E00E94DE2580E068
:10238000A881B9818C930C941612AAE7B0E04D9104
:102390005D916D917C91A6E7B0E00D911D912D911D
:1023A0003C910E94942711F00C94DC11AA85BB8506
:1023B0000E94E6250C941612EAECF0E0FA93EA93F8
:1023C0005A924A92AAECB0E00D911D912D913C9148
:1023D000A42DB52D0D931D932D933C9384E00E9465
:1023E000E2250E947D16249684E00E94DE25EA857F
:1023F000FB85FA93EA935A924A92AAECB0E00D91C7
:102400001D912D913C91A42DB52D0D931D932D93D0
:102410003C9384E00E94E2250E941316249684E0F7
:102420000E94DE2580E0A881B9818C930C941C1257
:10243000AA85BB850E94E6250027ACE6B0E08C911A
:1024400086FB0EF401E041E0041711F00C94211119
:10245000C49AA885B9850D911C91003050E01507EC
:1024600011F00C943B12A8EBB0E08D919C91A6EB7F
:10247000B0E08D939C930091D200013081E009F08F
:1024800080E08F930027A3EDB0E08C9186FB0EF4E3
:1024900001E040E0041781E009F080E09F9189238A
:1024A000882311F40C945F1280E593EC90934D0017
:1024B00080934C0081E08EBD89B7846089BF83E042
:1024C000481A8827580A2696089584E00E94032710
:1024D00084E00E94032781E00E94032781E00E949C
:1024E000032781E00E94032781E00E94032780E008
:1024F000AE81BF818C93AE81BF810C910F3018F0FB
:1025000011F00C94201481E0AC81BD818C93AC81DE
:10251000BD810C910C3018F011F00C94A7128FEFC4
:102520000E94E7260E94E9260E94E826AC81BD8130
:10253000AD90BB24A4E8B0E0AA0DBB1D8C93AC8188
:10254000BD818C918F5F8C9310F40C9487128DE079
:10255000AC81BD818C93AC81BD810C91043118F0AC
:1025600011F00C94C5128FEF0E94E7260E94E92615
:102570000E94E826A881B9818C93AC81BD818C91A1
:102580008F5F8C9310F40C94AB12EA85FB85FA9361
:10259000EA93EA85FB85FA93EA930E94A8142496AD
:1025A0000027ACE6B0E08C9186FB0EF401E041E040
:1025B000041711F00C94DE120C94181480E0AA8118
:1025C000BB818C9300919000003281E009F080E0A3
:1025D0008F9300919000003181E009F080E09F919D
:1025E000892B882311F40C94F91281E0AA81BB8114
:1025F0008C9300918500003081E009F480E08F9396
:1026000000918500053E81E009F480E09F918923D7
:102610008F93AA81BB810C91013081E009F080E0A9
:102620009F918923882311F40C940D14009190003C
:10263000003211F00C942013A8EBB0E00E94F525B5
:102640000027ACE6B0E08C9185FB0EF401E040E0A1
:10265000041711F00C94551381E0AC81BD818C936B
:10266000AC85BD854D915C91A8EBB0E00D911C91BE
:102670000417150781E009F080E08F93A8EBB0E024
:102680000D911C91003050E0150780E010F009F02A
:1026900081E09F918923882311F40C94531380E0E7
:1026A000AC81BD818C930C94891380E0AC81BD8199
:1026B0008C9381E0A881B9818C93A881B9810C9118
:1026C000053018F011F00C948913A881B981AD90F0
:1026D000BB24AFE9B0E0AA0DBB1D4C91A881B98124
:1026E000AD90BB24A4E8B0E0AA0DBB1D0C9104176B
:1026F00011F40C94811381E0AC81BD818C930C9416
:102700008913A881B9818C918F5F8C9310F40C94FC
:102710005D13AC81BD810C91003081E009F080E057
:102720008F93AC85BD850D911C910F315EE415072B
:1027300081E009F080E09F91892B882311F40C94AB
:102740000D140E943A14A885B9850D911D912D9103
:102750003C9140E052E060E070E00E947426A2E903
:10276000B0E04D935D936D937D93E6E9F0E0FA93CD
:10277000EA935A924A92AE85BF850D911D912D9193
:102780003C91A42DB52D0D931D932D933C9384E086
:102790000E94E2250E941316249684E00E94DE2502
:1027A0008091900080939100AC85BD850D911C9126
:1027B0000F315EE4150711F00C94DE13AC81BD817E
:1027C0000C91003011F00C940D1480916C00806419
:1027D00080936C0000919100003181E009F080E06D
:1027E0008F93AC85BD850D911C910F315EE415076B
:1027F00081E009F480E09F918923882311F40C94EF
:102800000D14AA85BB850D911D912D913C91AEECC7
:10281000B0E00D931D932D933C9300918500003003
:1028200011F00C94181480916C00806480936C00FB
:10283000AE81BF818C918F5F8C9310F40C947B12CE
:102840008FEF0E94E7260E94E9260E94E826A0E674
:10285000B0E08C938FEF0E94E7260E94E9260E9449
:10286000E826A0E6B0E08C938CE0481A8827580A46
:102870002C96089581E00E940327A8EAB0E08827FB
:102880008C9381E0A881B9818C93A881B9810C9146
:10289000083018F011F00C947414A881B981AD902F
:1028A000BB24A4E8B0E0AA0DBB1D0C91003211F4CA
:1028B0000C946C14A881B981AD90BB24A4E8B0E05D
:1028C000AA0DBB1D8C91A8EAB0E08F930E946426EC
:1028D0008F918D9388278C93A881B9818C918F5F7C
:1028E0008C9310F40C944514A8EAB0E00E9464267E
:1028F000E8ECF0E50E94362789E0A881B9818C9345
:10290000A881B9810C910B3018F011F00C94A2142D
:10291000A881B981AD90BB24A4E8B0E0AA0DBB1D8D
:102920008C91A8EAB0E08F930E9464268F918D93DA
:1029300088278C93A881B9818C918F5F8C9310F438
:102940000C94801481E0481A8827580A229608952A
:1029500081E00E94032781E00E94032784E00E9417
:1029600003278FEF0E94E7260E94E9260E94E826AF
:10297000AC81BD818C938FEF0E94E7260E94E926EF
:102980000E94E826AA81BB818C93AA81BB810C910D
:1029900011272227332740E051E060E070E00E94D9
:1029A0001327A885B9850D931D932D933D93A88575
:1029B000B9850D911D912D913C91AC81BD814C91BA
:1029C0005527662777270E948A27A885B9850D9302
:1029D0001D932D933D93A885B9850D911D912D9142
:1029E0003C9140E050E061E070E00E941327A88134
:1029F000B9810D931D932D933D938FEF0E94E72690
:102A00000E94E9260E94E826AC81BD818C938FEF5D
:102A10000E94E7260E94E9260E94E826AC81BD813B
:102A20008C938FEF0E94E7260E94E9260E94E826F9
:102A3000AC81BD818C938FEF0E94E7260E94E9262E
:102A40000E94E826AC81BD818C938FEF0E94E7261F
:102A50000E94E9260E94E826AC81BD818C938FEF0D
:102A60000E94E7260E94E9260E94E826AA81BB81EF
:102A70008C93AA81BB810C9111272227332740E038
:102A800051E060E070E00E941327A885B9850D939E
:102A90001D932D933D93A885B9850D911D912D9181
:102AA0003C91AC81BD814C915527662777270E94C8
:102AB0008A27A885B9850D931D932D933D93A885ED
:102AC000B9850D911D912D913C91A881B9814D91B0
:102AD0005D916D917C910E948A27A885B9850D939F
:102AE0001D932D933D938FEF0E94E7260E94E926C8
:102AF0000E94E826AC81BD818C938FEF0E94E7266F
:102B00000E94E9260E94E826AA81BB818C93AA81B3
:102B1000BB810C9111272227332740E051E060E070
:102B200070E00E941327A881B9810D931D932D9306
:102B30003D93A881B9810D911D912D913C91AC815E
:102B4000BD814C915527662777270E948A27A88147
:102B5000B9810D931D932D933D938FEF0E94E7262E
:102B60000E94E9260E94E826AC81BD818C938FEFFC
:102B70000E94E7260E94E9260E94E826AA81BB81DE
:102B80008C93AA81BB810C9111272227332740E027
:102B900051E060E070E00E941327AE81BF810D9389
:102BA0001D932D933D93AE81BF810D911D912D916C
:102BB0003C91AC81BD814C915527662777270E94B7
:102BC0008A27AE81BF810D931D932D933D93AE81D6
:102BD000BF810D911D912D913C9140E050E061E04D
:102BE00070E00E941327AE81BF810D931D932D933A
:102BF0003D93AE81BF810D911D912D913C91A88196
:102C0000B9814D915D916D917C910E948A27AE8131
:102C1000BF810D931D932D933D9386E0481A88271D
:102C2000580A2696089584E00E94032784E00E94B3
:102C30000327AC81BD810D911D912D913C9142E006
:102C400050E060E070E00E948F27A881B9810D9369
:102C50001D932D933D93A3E7B0E00C9111272227FC
:102C60003327A881B9814D915D916D917C910E942E
:102C70001327AA81BB810D931D932D933D93AA81A8
:102C8000BB810D911D912D913C91AAE7B0E04D9132
:102C90005D916D917C910E948A27AA81BB810D93E1
:102CA0001D932D933D93009182000B3011F40C94F1
:102CB0006B16AA81BB810D911D912D913C9140E233
:102CC00050E060E070E00E948A27AA81BB810D93EA
:102CD0001D932D933D93AA81BB810D911D912D9143
:102CE0003C91AE81BF810D931D932D933C9388E061
:102CF000481A8827580A2496089584E00E940327DA
:102D000082E00E940327009182000B3011F00C94A6
:102D1000C116AC81BD810D911D912D913C9140E872
:102D200050E060E070E00E947426A5EDB0E04D93A5
:102D30005D936D937D93AC81BD810D911C9140E8B5
:102D400050E00E944A26A881B9810D931C93A88166
:102D5000B9810D911C9144E050E00E940927A8819F
:102D6000B9810D931C93A881B9810D911C9144E008
:102D700050E0040F151FA881B9810D931C930C948A
:102D8000F716AC81BD810D911D912D913C9140E0D4
:102D900051E060E070E00E947426A5EDB0E04D9334
:102DA0005D936D937D93AC81BD810D911C9140E04D
:102DB00051E00E944A26A881B9810D931C93A881F5
:102DC000B9810D911C9142E050E00E940927A88131
:102DD000B9810D931C93A881B9810D911C9142E09A
:102DE00050E0040F151FA881B9810D931C93A5ED28
:102DF000B0E00D911D912D913C91AEE7B0E04D9169
:102E00005D916D917C910E948A27A5EDB0E00D93B4
:102E10001D932D933D93A5EDB0E00D911D912D9146
:102E20003C91A1E7B0E04D915C91662777270E9425
:102E30008A27A5EDB0E00D931D932D933D930E943D
:102E4000CD1EA881B981AD90BC90ADEDB0E0AA0DCA
:102E5000BB1D8C91AA81BB818D9388278D938D9307
:102E60008C93A881B9810E94FC25AA81BB810D9118
:102E70001D912D913C9140E051E060E070E00E9496
:102E80001327AA81BB810D931D932D933D93AA8196
:102E9000BB810D911D912D913C91A881B981AD907F
:102EA000BC90ADEDB0E0AA0DBB1D4C915527662737
:102EB00077270E948A27AA81BB810D931D932D93AA
:102EC0003D93009182000B3011F00C94C717A8813C
:102ED000B9810E94FC25AA81BB810D911D912D9184
:102EE0003C9140E051E060E070E00E941327AA812D
:102EF000BB810D931D932D933D93AA81BB810D91B1
:102F00001D912D913C91A881B981AD90BC90ADED02
:102F1000B0E0AA0DBB1D4C915527662777270E946C
:102F20008A27AA81BB810D931D932D933D93A88180
:102F3000B9810E94FC25AA81BB810D911D912D9123
:102F40003C9140E051E060E070E00E941327AA81CC
:102F5000BB810D931D932D933D93AA81BB810D9150
:102F60001D912D913C91A881B981AD90BC90ADEDA2
:102F7000B0E0AA0DBB1D4C915527662777270E940C
:102F80008A27AA81BB810D931D932D933D93AA811E
:102F9000BB810D911D912D913C91AE81BF810D930F
:102FA0001D932D933C9386E0481A8827580A24964F
:102FB000089580E0A881B9818C930027BB27A0E306
:102FC0008C9183FB0EF401E040E0041711F00C94A7
:102FD000ED1782E0A881B9818C930027BB27A0E37D
:102FE0008C9184FB0EF401E040E0041711F00C9486
:102FF000FD1781E0A881B9818C930027BB27A3E34B
:103000008C9181FB0EF401E040E0041711F00C9468
:103010000D1883E0A881B9818C930027BB27A3E317
:103020008C9181FB0EF401E040E0041781E009F08F
:1030300080E08F930027BB27A0E38C9183FB0EF4E5
:1030400001E040E0041781E009F080E09F918923CE
:10305000882311F40C94301884E0A881B9818C93F2
:10306000089581E00E94032781E00E94032782E007
:103070000E9403275398549880E081BB909A919ABC
:10308000EF93FF93E0EFF1E00E94C826FF91EF91EC
:1030900080E0AC81BD818C930027BB27A0E38C919D
:1030A00080FB0EF401E040E0041711F00C945C1872
:1030B00081E0AC81BD818C930027BB27A0E38C917C
:1030C00081FB0EF401E040E0041711F00C946D1840
:1030D000AC81BD818C918E5F8C930027BB27A9E3C7
:1030E0008C9185FB0EF401E040E0041711F00C9484
:1030F0007E18AC81BD818C918C5F8C930027BB279F
:10310000A9E38C9184FB0EF401E040E0041711F078
:103110000C948F18AC81BD818C91885F8C93AC81AD
:10312000BD810C91003018F011F00C9499180C949A
:10313000F21885E090E00E94F42680E0AA81BB812D
:103140008C930027BB27A0E38C9180FB0EF401E059
:1031500040E0041711F00C94B11881E0AA81BB8102
:103160008C930027BB27A0E38C9181FB0EF401E038
:1031700040E0041711F00C94C218AA81BB818C9115
:103180008E5F8C930027BB27A9E38C9185FB0EF4FF
:1031900001E040E0041711F00C94D318AA81BB8120
:1031A0008C918C5F8C930027BB27A9E38C9184FBC7
:1031B0000EF401E040E0041711F00C94E418AA8129
:1031C000BB818C91885F8C93AA81BB814C91AC812F
:1031D000BD810C91041711F40C94F21880E0AC81BD
:1031E000BD818C93AC81BD810C91033011F00C94A6
:1031F000FF1882E0AC81BD818C930C943519AC81B1
:10320000BD810C91043081E008F480E08F93AC81A3
:10321000BD810C91073081E010F009F080E09F91B2
:103220008923882311F40C941B1983E0AC81BD81A0
:103230008C930C943519AC81BD810C91083081E0E0
:1032400008F480E08F93AC81BD810C910F3081E058
:1032500010F009F080E09F918923882311F40C94E9
:10326000351984E0AC81BD818C9381E081BB91985C
:10327000539A549AAC81BD818C91AE81BF818C935D
:1032800084E0481A8827580A2696089581E00E940B
:10329000032781E00E940327AC81BD818C91A88126
:1032A000B9818C930E94F30888EC90E00E94F42688
:1032B0005A924A9281E0A42DB52D8C9381E00E9410
:1032C000E2250E944323229681E00E94DE25A895F4
:1032D000EBE6F0E0FA93EA930E94D91722968AE08F
:1032E00090E00E94F42600916B00003011F00C94E5
:1032F000671986E990E00E94F4265A924A9280E08B
:10330000A42DB52D8C9381E00E94E2250E944323D9
:10331000229681E00E94DE2584E690E00E94F42659
:103320005A924A9280E0A42DB52D8C9381E00E94A0
:10333000E2250E944323229681E00E94DE25A89583
:10334000EBE6F0E0FA93EA930E94D91722960E94E6
:10335000F5085A924A9281E0A42DB52D8C9381E014
:103360000E94E2250E944323229681E00E94DE25EE
:1033700084E690E00E94F4265A924A9280E0A42DBE
:10338000B52D8C9381E00E94E2250E944323229672
:1033900081E00E94DE258AE090E00E94F4265A92A5
:1033A0004A9280E0A42DB52D8C9381E00E94E22505
:1033B0000E944323229681E00E94DE250E94F308AA
:1033C00086E990E00E94F42600916B00003018F02E
:1033D00011F00C94ED190C949F1988E790E00E946D
:1033E000F4265A924A9281E0A42DB52D8C9381E067
:1033F0000E94E2250E94041B229681E00E94DE25A5
:10340000A881B9810C91023011F00C94471A0091F7
:103410006B00013011F00C94121A81E08093C5000A
:103420000C94401A023011F00C942A1A80E0809318
:10343000C5005A924A9281E0A42DB52D8C9381E06B
:103440000E94E2250E94041B229681E00E94DE2554
:103450000C94401A033011F00C94401A83E08093CE
:10346000C5005A924A9282E0A42DB52D8C9381E03A
:103470000E94E2250E94041B229681E00E94DE2524
:10348000EEE0F0E0A5ECB0E07BE70E941D28A8810B
:10349000B9810C91033011F00C94701A00916B00FB
:1034A000013011F00C94591A81E0809370000C9453
:1034B000691A023011F00C94621A80E08093700057
:1034C0000C94691A033011F00C94691A82E080930D
:1034D0007000E1E1F0E0A0E7B0E07BE70E941D288A
:1034E000A881B9810C91013011F00C94C21A00919D
:1034F0006B00013011F00C94891AA6ECB0E08C91AD
:10350000897F8C93A6ECB0E08C9182608C930C94B4
:10351000BB1A023011F00C94A31AA6ECB0E08C9107
:10352000897F8C935A924A9281E0A42DB52D8C9379
:1035300081E00E94E2250E94041B229681E00E9405
:10354000DE250C94BB1A033011F00C94BB1AA6ECC8
:10355000B0E08C9186608C935A924A9284E0A42DBC
:10356000B52D8C9381E00E94E2250E94041B2296D7
:1035700081E00E94DE25EFE0F0E0A6ECB0E07BE722
:103580000E941D280E94F708A895EBE6F0E0FA9348
:10359000EA930E94D917229685E090E00E94F426D3
:1035A00000916B00003011F00C94C41A86E990E091
:1035B0000E94F4265A924A9280E0A42DB52D8C9355
:1035C00081E00E94E2250E944323229681E00E942E
:1035D000DE2586E990E00E94F4265A924A9280E025
:1035E000A42DB52D8C9381E00E94E2250E944323F7
:1035F000229681E00E94DE250E94F50882E0481AAA
:103600008827580A2496089581E00E94032781E0C4
:10361000A881B9818C93AA81BB814C91A881B98181
:103620000C91041718F011F00C94311B5A924A9225
:1036300082E0A42DB52D8C9381E00E94E2250E94AA
:103640004323229681E00E94DE258DE790E00E94D0
:10365000F426A881B9818C918F5F8C9310F40C941F
:103660000B1B81E0481A8827580A2296089581E0AA
:103670000E94032781E0A881B9818C93A881B98138
:103680000C91063018F011F00C945A1B0E94F308AC
:103690008FE090E00E94F4260E94F50884E690E016
:1036A0000E94F426A881B9818C918F5F8C9310F4CD
:1036B0000C943E1B81E0481A8827580A22960895E8
:1036C0000E94E026C39A88EC90E00E94F42681B51F
:1036D000886081BD0E9405225A924A9281E0A42D01
:1036E000B52D8C9381E00E94E2250E945122229602
:1036F00081E00E94DE2581B5886181BD877F81BD23
:1037000084E690E00E94F426FF27E0E1FA93EA9332
:103710005A924A928BE0A42DB52D8C9381E00E94A1
:10372000E2250E94E824249681E00E94DE250130F3
:1037300051E0150711F00C94B01B5A924A92A0EC7C
:10374000B0E08D919C91A42DB52D8D939C9382E03A
:103750000E94E2250E94E922229682E00E94DE2554
:103760005A924A9282E3A42DB52D8C9381E00E9457
:10377000E2250E945122229681E00E94DE25C29A13
:10378000D89A82E390E00E94F426089581E00E9496
:10379000032781E00E9403278FEFAA81BB818C93CE
:1037A00080E0A881B9818C93A881B9810C910F30F8
:1037B00018F011F00C94E91B91E0AA81BB810E94E2
:1037C000D626A881B9818C918F5F8C9310F40C94CC
:1037D000D41B82E0481A8827580A2496089581E06D
:1037E0000E94032781E00E94032781E00E940327B3
:1037F00082E00E94032782E00E9403278FEFAA85C0
:10380000BB858C93C49A0E94C61BC498EE81FF812D
:10381000FA93EA935A924A9280E4A42DB52D8C93A0
:1038200081E00E94E2255A924A9200E010E020E0F6
:1038300030E0A42DB52D0D931D932D933C9384E082
:103840000E94E2250E947921269685E00E94DE25CD
:10385000AE81BF810C91013011F40C94321CC49ADA
:103860000C94C71E81E0AA85BB858C9380E293E00F
:10387000A881B9818D939C93EE81FF81FA93EA939D
:103880005A924A9287E7A42DB52D8C9381E00E942D
:10389000E2255A924A9200E010E020E030E0A42DA8
:1038A000B52D0D931D932D933C9384E00E94E2254A
:1038B0000E947921269685E00E94DE2581E090E035
:1038C0000E94F426EE81FF81FA93EA935A924A927B
:1038D00089E6A42DB52D8C9381E00E94E2255A92B1
:1038E0004A9200E010E020E030E0A42DB52D0D93C9
:1038F0001D932D933C9384E00E94E2250E94792140
:10390000269685E00E94DE2581E090E00E94F42664
:10391000AE81BF810C91003081E009F080E08F938F
:10392000AE81BF810C91053081E009F080E09F916C
:10393000892B8F93A881B9810D911C91003050E0A3
:10394000150781E009F080E09F91892B882311F40D
:103950000C943C1CAE81BF810C91003011F00C9492
:10396000B41CC49A0C94111D80E293E0A881B98123
:103970008D939C93EE81FF81FA93EA935A924A9237
:1039800081E4A42DB52D8C9381E00E94E2255A920A
:103990004A9200E010E020E030E0A42DB52D0D9318
:1039A0001D932D933C9384E00E94E2250E9479218F
:1039B000269685E00E94DE25A881B9810D911C9193
:1039C00041E050E0041B150BA881B9810D931C93B5
:1039D00081E090E00E94F426AE81BF810C9100301E
:1039E00081E009F080E08F93A881B9810D911C914D
:1039F000003050E0150781E009F080E09F91892BAD
:103A0000882311F40C94BA1CC49AA881B9810D9131
:103A10001C91003050E0150711F00C94111D0C940E
:103A2000C71E8AE090E00E94F426C498EE81FF81D0
:103A3000FA93EA935A924A9280E5A42DB52D8C937D
:103A400081E00E94E2255A924A9201E010E020E0D3
:103A500030E0A42DB52D0D931D932D933C9384E060
:103A60000E94E2250E947921269685E00E94DE25AB
:103A7000C49A82E390E00E94F42600E010E020E087
:103A800030E0AEE7B0E00D931D932D933C9300E042
:103A900010E020E030E0A5EDB0E00D931D932D93F4
:103AA0003C930E94CD1E00E010E020E030E0A5ED48
:103AB000B0E00D931D932D933C930027A3EDB0E050
:103AC0008C9186FB0EF401E041E0041711F00C9498
:103AD0006B1D0C94C71E0091EA00023011F40C9487
:103AE000FE1D8091A00280938200A7EAB2E00D91B2
:103AF000112740E051E00E940927AA81BB810D9364
:103B00001C93AA81BB810D911C91A6EAB2E04D9154
:103B10005527040F151FAA81BB810D931C93AA8101
:103B2000BB810D911C912227332740E050E061E0DA
:103B300070E00E941327AEE7B0E00D931D932D9324
:103B40003D93A5EAB2E00D91112740E051E00E94BB
:103B50000927AA81BB810D931C93AA81BB810D917A
:103B60001C91A4EAB2E04D915527040F151FAA81BC
:103B7000BB810D931C93AEE7B0E00D911D912D918B
:103B80003C91AA81BB814D915C91662777270E9469
:103B90008A27AEE7B0E00D931D932D933D930091DE
:103BA00082000C3011F00C94D81D8BE080938200C1
:103BB000009182000E3011F00C94E11D8BE0809397
:103BC0008200009182000F3011F00C94EA1D8BE00E
:103BD00080938200AEE7B0E00D911D912D913C9154
:103BE000A5EDB0E00D931D932D933C930E94CD1E47
:103BF000A5EDB0E00E9403260C94101E0091140164
:103C0000063411F00C94071E84E08093820000912A
:103C10003001063411F00C94101E8BE0809382006A
:103C2000A8958091EB0080937300009173000030A1
:103C300011F00C941D1E0C94C71E009173000034EB
:103C400018F011F00C94261E0C94281E0C94C71E1C
:103C50008091EC00AE81BF818C938091ED00AC81AE
:103C6000BD818C93AC81BD819C91AE81BF818C91D3
:103C7000A1E7B0E08D939C938091F400AE81BF8169
:103C80008C938091F500AC81BD818C93AC81BD811A
:103C90009C91AE81BF818C91A4E7B0E08D939C9301
:103CA000A4E7B0E00D911C91003050E0150711F031
:103CB0000C94701E80910201AE81BF818C93809123
:103CC0000301AC81BD818C93AC81BD819C91AE819F
:103CD000BF818C91A4E7B0E08D939C930C94701EEF
:103CE000A895A4E7B0E00D911C91003050E01507B5
:103CF00011F00C947D1E0C94C71E02E010E020E031
:103D000030E0A4E7B0E04D915C91662777270E94F0
:103D10001327A6E7B0E00D931D932D933D93A6E7DF
:103D2000B0E00D911D912D913C91A1E7B0E04D9136
:103D30005C91662777270E948A27A6E7B0E00D935B
:103D40001D932D933D93A6E7B0E00D911D912D910C
:103D50003C91A5EDB0E04D915D916D917C910E94FB
:103D60008A27A6E7B0E00D931D932D933D93A6E718
:103D7000B0E00D911D912D913C91A5EDB0E00D931A
:103D80001D932D933C9380E0AA85BB858C9387E09F
:103D9000481A8827580A2A96089581E00E94032726
:103DA00081E00E94032782E00E94032782E00E94B4
:103DB00003278FEFAE81BF818C9391E0AE81BF81ED
:103DC0000E94D62691E0AE81BF810E94D62691E066
:103DD000AE81BF810E94D62691E0AE81BF810E9454
:103DE000D62691E0AE81BF810E94D62691E0AE81B9
:103DF000BF810E94D62691E0AE81BF810E94D62667
:103E000091E0AE81BF810E94D62691E0AE81BF8154
:103E10000E94D62691E0AE81BF810E94D62691E015
:103E2000AE81BF810E94D62691E0AE81BF810E9403
:103E3000D62691E0AE81BF810E94D62691E0AE8168
:103E4000BF810E94D62691E0AE81BF810E94D62616
:103E500091E0AE81BF810E94D626C49880E090E0B8
:103E6000A881B9818D939C938FEF0E94E7260E94D1
:103E7000E9260E94E826AE81BF818C93A881B98192
:103E80000E94F525AE81BF810C91003081E009F4DC
:103E900080E08F93A881B9810D911C91003050E092
:103EA000150781E009F080E09F91892B882311F4A8
:103EB0000C94341FA881B9810D911C91003050E001
:103EC000150711F00C946B1F8091D30080648093D0
:103ED000D3000C949020EE81FF81FA93EA935A92DA
:103EE0004A9281E5A42DB52D8C9381E00E94E225B4
:103EF0005A924A92A5EDB0E00D911D912D913C9101
:103F0000A42DB52D0D931D932D933C9384E00E9419
:103F1000E2250E947921269685E00E94DE25002771
:103F2000A3EDB0E08C9186FB0EF401E041E00417B4
:103F300011F00C949D1F0C949020A895AE81BF8128
:103F40000C91003011F00C94E21F80E090E0A88109
:103F5000B9818D939C938FEF0E94E7260E94E926FA
:103F60000E94E826AE81BF818C93A881B9810E940E
:103F7000F525AE81BF810C91003081E009F480E02D
:103F80008F93A881B9810D911C91003050E01507E5
:103F900081E009F080E09F91892B882311F40C9433
:103FA000AB1FA881B9810D911C91003050E015071D
:103FB00011F00C94E21F8091D30080648093D300B1
:103FC0000C949020AE81BF810C910F3F11F00C94A6
:103FD000262080E090E0A881B9818D939C938FEF9B
:103FE0000E94E7260E94E9260E94E826AE81BF8152
:103FF0008C93A881B9810E94F525AE81BF810C9177
:104000000F3F81E009F480E08F93A881B9810D9181
:104010001C91003050E0150781E009F080E09F918D
:10402000892B882311F40C94EF1FA881B9810D917D
:104030001C91003050E0150711F00C94262080915F
:10404000D30080648093D3000C949020AE81BF8114
:104050000C910E3F11F40C943520C49A8091D3003A
:1040600080648093D3000C94902080E090E0AA813B
:10407000BB818D939C9380E0AE81BF818C93AE8198
:10408000BF810C910F3F18F011F00C947720AA819A
:10409000BB810E94F5258FEF0E94E7260E94E9264A
:1040A0000E94E826AA81BB81AD90BC90ADEDB0E046
:1040B000AA0DBB1D8C93AA81BB810E94F5258FEFB1
:1040C0000E94E7260E94E9260E94E826AA81BB8179
:1040D000AD90BC90ADEDB0E0AA0DBB1D8C93AE8150
:1040E000BF818C918F5F8C9310F40C943F208FEFE5
:1040F0000E94E7260E94E9260E94E826AE81BF8141
:104100008C938FEF0E94E7260E94E9260E94E82602
:10411000AE81BF818C93C49AA5EDB0E00E94E625E4
:1041200086E0481A8827580A2896089582E00E9457
:10413000032781E00E94032780E0AE81BF818C933A
:104140000E94C61BC49880E090E0AA81BB818D9339
:104150009C938FEF0E94E7260E94E9260E94E826A2
:10416000A881B9818C93AA81BB810E94F525A8956D
:10417000A881B9810C91003081E009F480E08F932F
:10418000AA81BB810D911C91003050E0150781E0A0
:1041900009F080E09F91892B882311F40C94A920C9
:1041A000AA81BB810D911C91003050E0150711F0E0
:1041B0000C94E1208091D30080648093D3000C9410
:1041C0007321E881F981FA93EA935A924A9281E540
:1041D000A42DB52D8C9381E00E94E2255A924A923B
:1041E000AA85BB850D911D912D913C91A42DB52DD6
:1041F0000D931D932D933C9384E00E94E2250E9431
:104200007921269685E00E94DE25A881B9810C914E
:10421000003011F00C94392180E090E0AA81BB813C
:104220008D939C938FEF0E94E7260E94E9260E94BF
:10423000E826A881B9818C93AA81BB810E94F525CB
:10424000A895A881B9810C91003081E009F480E043
:104250008F93AA81BB810D911C91003050E015070E
:1042600081E009F080E09F91892B882311F40C9460
:104270001221A881B9810C910F3F11F00C946D218E
:1042800080E090E0AA81BB818D939C938FEF0E9488
:10429000E7260E94E9260E94E826A881B9818C932E
:1042A000AA81BB810E94F525A895A881B9810C91AE
:1042B0000F3F81E009F480E08F93AA81BB810D91CB
:1042C0001C91003050E0150781E009F080E09F91DB
:1042D000892B882311F40C944621A881B9818C91F3
:1042E000AE81BF818C9383E0481A8827580A2496B0
:1042F000089584E00E94032781E00E94032782E062
:104300000E9403278FEFAA81BB818C9391E0AA8141
:10431000BB810E94D62691E0A885B9850E94D62649
:10432000AE81BF810D911D912D913C9140E052E0F5
:1043300060E070E00E941327AC81BD810D931D9356
:104340002D933D93AC81BD818F9314968E910E94E5
:10435000FA218E910E94FA218E910E94FA218E916B
:104360000E94FA2185E90E94FA218F9180E090E075
:10437000A881B9818D939C938FEF0E94E7260E94BC
:10438000E9260E94E826AA81BB818C93A881B98185
:104390000E94F525A895AA81BB810C910F3F81E071
:1043A00009F480E08F93A881B9810D911C910030B0
:1043B00050E0150781E009F080E09F91892B882368
:1043C00011F40C94BC21A881B9810D911C9100308D
:1043D00050E0150711F00C94F2218091D300806415
:1043E0008093D300AA81BB818C91AA85BB858C93D5
:1043F0000C94FF218FB9779BFECF8FB1089587E092
:10440000481A8827580A269608955A924A9284E2B2
:1044100098E0A42DB52D8D939C9382E00E94E22517
:104420005A924A9280E0A42DB52D8C9381E00E948F
:10443000E2250E948D24249683E00E94DE25EF93DE
:10444000FF93ECE8F1E00E94C826FF91EF91BB27B3
:10445000A0E38C9182FBDEF782E090E00E94F426DC
:104460005A924A9280E298E0A42DB52D8D939C93A8
:1044700082E00E94E2255A924A9280E0A42DB52D56
:104480008C9381E00E94E2250E948D24249683E093
:104490000E94DE2582E090E00E94F4260E9406231E
:1044A000089582E00E94032700E011E0AA81BB8109
:1044B0004D9155270E940927A881B9810D931C931E
:1044C000A881B9810D911C91AA81BB814D9155277D
:1044D000040F151FA881B9810D931C935A924A921B
:1044E000AA81BB818D919C91A42DB52D8D939C9318
:1044F00082E00E94E2255A924A928BE0A42DB52DCB
:104500008C9381E00E94E2250E948D24249683E012
:104510000E94DE255A924A9280E298E0A42DB52DA1
:104520008D939C9382E00E94E2255A924A9280E009
:10453000A42DB52D8C9381E00E94E2250E948D244C
:10454000249683E00E94DE2582E0481A8827580AD4
:104550002296089582E00E94032700E110E0AC81DA
:10456000BD814D9155270E940927A881B9810D93DE
:104570001C93A881B9810D911C91AA81BB814D9199
:104580005527040F151FA881B9810D931C935A92CA
:104590004A92AA81BB818D919C91A42DB52D8D93BA
:1045A0009C9382E00E94E2255A924A9282E0A42DD6
:1045B000B52D8C9381E00E94E2250E948D242496E3
:1045C00083E00E94DE2582E0481A8827580A229656
:1045D00008955A924A92AA81BB818D919C91A42DF3
:1045E000B52D8D939C9382E00E94E2255A924A92C7
:1045F00083E0A42DB52D8C9381E00E94E2250E94DA
:104600008D24249683E00E94DE25089581E00E9497
:10461000032781E00E940327C49AD898C29880E0BB
:10462000A881B9818C9380E0AA81BB818C93AA81F7
:10463000BB810C910F3118F011F00C943B2391E0E9
:10464000A881B9810E94D62691E0A881B9810E94F3
:10465000D62691E0A881B9810E94D62691E0A88152
:10466000B9810E94D626AA81BB818C918F5F8C93E1
:1046700010F40C941723C29AD89A82E0481A88271B
:10468000580A2496089581E00E9403275A924A927C
:1046900080E298E0A42DB52D8D939C9382E00E943A
:1046A000E2255A924A9280E0A42DB52D8C9381E0A8
:1046B0000E94E2250E948D24249683E00E94DE253C
:1046C000AA81BB810C91003011F00C9476235A9290
:1046D0004A9280E0A42DB52D8C9381E00E94E225C2
:1046E0000E94F023229681E00E94DE25AA81BB81F0
:1046F0000C91013011F00C948C235A924A9285E669
:10470000A42DB52D8C9381E00E94E2250E94F02318
:10471000229681E00E94DE25AA81BB810C910230A5
:1047200011F00C94B9235A924A9283E6A42DB52D28
:104730008C9381E00E94E2250E94F023229681E082
:104740000E94DE2588EC90E00E94F4265A924A925C
:1047500080E0A42DB52D8C9381E00E94E2250E947B
:10476000F023229681E00E94DE2582E390E00E9401
:10477000F426AA81BB810C91033011F00C94E22342
:104780005A924A9282E6A42DB52D8C9381E00E9424
:10479000E2250E94F023229681E00E94DE2580E936
:1047A00091E00E94F4265A924A9280E0A42DB52D01
:1047B0008C9381E00E94E2250E94F023229681E002
:1047C0000E94DE258AE090E00E94F4268AE090E0D4
:1047D0000E94F42681E0481A8827580A22960895F4
:1047E00081E00E940327C49A5A924A928CE3A42D36
:1047F000B52D8C9381E00E94E2250E9451222296E1
:1048000081E00E94DE25D898C298AA81BB810C91D4
:10481000003018F011F00C940F240C94492483E517
:10482000A881B9818C9391E0A881B9810E94D62694
:104830008FEEA881B9818C9391E0A881B9810E9403
:10484000D6268EE6A881B9818C9391E0A881B981A2
:104850000E94D62691E0AA81BB810E94D62680E0E4
:10486000A881B9818C9391E0A881B9810E94D62654
:1048700091E0A881B9810E94D62691E0A881B981F2
:104880000E94D62691E0A881B9810E94D6260C9478
:10489000852485E4A881B9818C9391E0A881B981B0
:1048A0000E94D62688E7A881B9818C9391E0A881DF
:1048B000B9810E94D62689E6A881B9818C9391E0BE
:1048C000A881B9810E94D62684E7A881B9818C93FA
:1048D00091E0A881B9810E94D62680E0A881B981A3
:1048E0008C9391E0A881B9810E94D62691E0A8819D
:1048F000B9810E94D62691E0A881B9810E94D6266E
:1049000091E0A881B9810E94D626C29AD89A81E006
:10491000481A8827580A2296089581E00E940327A2
:10492000C29AD8985A924A9282E0A42DB52D8C93BF
:1049300081E00E94E2250E944225229681E00E94A9
:10494000DE255A924A92AC81BD818C91A42DB52D61
:104950008C9381E00E94E2250E944225229681E00C
:104960000E94DE25AC81BD8111968C91A881B98110
:104970008C935A924A92AA81BB818C91A42DB52D19
:104980008C9381E00E94E2250E944225229681E0DC
:104990000E94DE25AC81BD818C91A881B9818C9368
:1049A0005A924A92AA81BB818C91A42DB52D8C93E9
:1049B00081E00E94E2250E944225229681E00E9429
:1049C000DE25D89A81E0481A8827580A2296089549
:1049D00081E00E94032781E00E94032782E00E9479
:1049E0000327C29AD8985A924A9283E0A42DB52DF3
:1049F0008C9381E00E94E2250E944225229681E06C
:104A00000E94DE255A924A92A885B9858C91A42DE0
:104A1000B52D8C9381E00E94E2250E9442252296CA
:104A200081E00E94DE25EC81FD81FA93EA930E94E9
:104A300048252296EA81FB81FA93EA930E94482551
:104A40002296D89AAC81BD810D91112740E051E0AA
:104A50000E940927A881B9810D931C93A881B9816F
:104A60000D911C91AA81BB814D915527040F151FF3
:104A7000A885B9850D931C9384E0481A8827580AA5
:104A80002696089591E0A881B9810E94D6260895BE
:104A900081E00E94032791E0A881B9810E94CB2682
:104AA000A881B9818C91AA81BB818C9381E0481A3D
:104AB0008827580A2296089582E00E94032781E001
:104AC0000E940327C49ABB27A0E38C9182FBDEF7E8
:104AD000C298AC81BD810D911C91003052E0150748
:104AE00011F00C94AB2581E090E0AA81BB818D93FD
:104AF0009C9380E0A881B9818C93A881B9810C91A5
:104B00000F3018F011F00C94A925BB27A0E38C916D
:104B100082FBDEF790E2AA81BB81AD90BC90ADED47
:104B2000B0E0AA0DBB1D0E94D626AA81BB810D91C3
:104B30001C9140E250E0040F151FAA81BB810D9328
:104B40001C93A881B9818C918F5F8C9310F40C9485
:104B50007D250C94D72581E090E0AA81BB818D93BF
:104B60009C93AC81BD814D915C91AA81BB810D91DB
:104B70001C910417150718F011F00C94D725BB27CA
:104B8000A0E38C9182FBDEF7C29A91E0AA81BB81FF
:104B9000AD90BC90ADEDB0E0AA0DBB1D0E94D62635
:104BA000AA81BB810E94F52510F40C94B125C29A0C
:104BB00083E0481A8827580A24960895481A8827B7
:104BC000580A0895480E8827581E08950D911D9182
:104BD0002D913C9181E0080F8827181F281F381F4E
:104BE0003C932E931E930E930895ED91FC91EF5FED
:104BF000FF4FFC93EE930895ED91FC91E150F0404E
:104C0000FC93EE9308950D911D912D913C910150CF
:104C10001040204030403C932E931E930E930895F5
:104C20004091DF025091E0020DE815E30E94242636
:104C300049E156E3040F151F0093DF021093E002D1
:104C4000498158810C944A2609D00E94092700FC0A
:104C500010D0089503D01ED001F8F9CF0024E894B5
:104C600057FF02C009D0689400F80BD010F8012457
:104C7000089502D009D00895509540954F5F5F4F39
:104C80000895E89417FF0895009510950F5F1F4F42
:104C900068940895352F242FE894452B11F46894D7
:104CA0000895512F402F0027112780E1440F551FF1
:104CB000001F111F021B130B416018F4020F131F7A
:104CC0004E7F8A9599F708958F938D918823E9F700
:104CD00011978F91089588EE93E086D03197D9F798
:104CE000089500FC05D0089530D005D001F8F9CF23
:104CF00037D03FD00895842F952FA62FB72FE89453
:104D0000452B462B472B11F468940895402F512FC3
:104D1000622F732F0027112722273327F0E2440F39
:104D2000551F661F771F001F111F221F331F081BEF
:104D3000190B2A0B3B0B416028F4080F191F2A1F7F
:104D40003B1F4E7FFA9559F708950024E89477FFAA
:104D500002C006D0689400F809D010F80124089524
:104D600012D04F5F5F4F6F4F7F4F0895E89437FF2A
:104D7000089500951095209530950F5F1F4F2F4F88
:104D80003F4F6894089540955095609570950895AB
:104D90003197F1F708950E94E7268C910E94E92649
:104DA0008D939A95D1F70E94E82608950E94E726F0
:104DB0008D910E94E9269A95D9F70E94E8260895D8
:104DC000BF9ABE98C69ABD9A80E58DB90895089598
:104DD00008958FB9779BFECF8FB10895689462F8DC
:104DE0000895E89462F80895EF93FF93EE27E82B77
:104DF000E92B31F0E0EDF7E03197F1F70197D1F7CA
:104E0000FF91EF9108955A924A92480E8827581EB2
:104E100008950F92B801469F8001479F100D569F3D
:104E2000100D0F9008950F921F922F92C801D90173
:104E3000489F80014A9F90014B9F202C499F100D55
:104E4000211D321D5A9F202C589F100D211D321DEF
:104E5000599F200D311D689F200D311D699F300D18
:104E6000789F300D2F901F900F9008950E943C273F
:104E70000D920020D9F70895C89531960020089525
:104E8000819104D08D938823D9F70895813618F045
:104E90008B3708F48F7D08952E2E3F2E9927819110
:104EA0008D3209F093958823D1F79A95E22DF32D51
:104EB000112361F0091718F011F0101B01C0191B24
:104EC00028F021F080E28D931A95E9F780818D32E8
:104ED00019F48D93319604C0222311F08BE28D9347
:104EE000091738F031F0091B21F080E38D930A9502
:104EF000E9F781918D938823E1F7332351F0EA2F6D
:104F0000FB2F319633958E9182933A95E1F78EE29D
:104F10008C930895040F151F261F371F0895041B37
:104F2000150B260B370B08950417150726073707AF
:104F30000895000F111F221F331F0895009510952B
:104F4000209530950F5F1F4F2F4F3F4F08950191D0
:104F500010810EC001911191219130810BC00191FE
:104F6000108117FF05C03FEF2FEF04C0008111270C
:104F70002227332737FF03C0E1DF8DE28D93CF93E4
:104F8000DF93CF92DF92EF92AA24BB24CC24DD24BE
:104F9000EE2440E2CAE0DD2755E093E38881890FE3
:104FA00087FD9F7083FD907F891B89935A95A9F790
:104FB000C0DFAA1CBB1CCC1CDD1CEE1C4A9551F7A3
:104FC000E894EFE0FF2782910ED0EB30E0F71EF07F
:104FD00068948A2D0CD088278D93EF90DF90CF9026
:104FE000DF91CF910895982F829501D0892F8F70EE
:104FF000805D26F0803309F4089568948D930895B8
:1050000088278D93089581918D938823E1F70895E2
:1050100009919191992351F08A95D9F7319781910E
:105020008D930A9519F08823D1F70895E9CFE19976
:10503000FECFEEBBFFBB3196089591E001C092E038
:105040007B3751F47FB7F894F2DF8D918DBBE29AF4
:10505000E19A9A95C9F77FBF7727089591E001C03B
:1050600092E0E5DFE09A8DB38D939A95D1F708959C
:10507000FF93881BF9E0001FFA9511F4FF91089542
:10508000881F841B18F4840F8894F5CF0894F3CFFD
:10509000689401C0E894AF93BF938D9116F09191FD
:1050A00003C00E943C27902D891718F011F4882323
:1050B000A1F7BF91AF9108954F005A0059004200E7
:0A50C000434F4E46494700002E0002
:00000001FF
